:1000000009C02CC00DC00DC00BC00AC077C07AC09B
:1000100007C09FC011241FBECFE9CDBFA6D0BFC06F
:10002000EFCF10E019BE00E044241895282F912F3F
:10003000812F887321F4812F8770821731F480E833
:100040008FBD82E883BF80EC8FBD9095907629F4B8
:10005000C59884E088BF8EE089BF089582B709B64D
:1000600001FE45C087FF47C012BE90E09595879579
:10007000382E9695879589BD8AE088BF89BF912FD4
:100080009F5F192F892F8095837009F41C7F84E06E
:10009000CDDF88E086BF802F002391F08150082FAC
:1000A00079F4912F20E016FF02C0146009C013FDFF
:1000B00006C09BE0941510F4186002C01B7F442416
:1000C000822D8F5F282EB9F488ED86B9212F912FCC
:1000D00016FF04C0842D8C3308F4439493FF0BC0A7
:1000E000842D8150482E39F4122F137F04C012BE84
:1000F00082E088BF89BF80E48ABF1895C59A8AE0EC
:1001000089BF189589B58034E0F487E284BB39BC97
:1001100000C0B39B09C0812F16FF0DC08F7B182F25
:1001200082FD08C000E007C0812F16FD04C0806476
:10013000182F177F02E3B49B02C01F7E07C0106117
:1001400005C085E073DF89B5885F86BF8FE384BB18
:10015000189595B116B8812F15FF04C09E3720F46D
:100160001F7D02C097FD1062189520E826BD81E032
:1001700086BD89E188BB80EC8FBD82E883BF91E2B8
:1001800097BB82E285BF80E48BBF8FE384BB28B935
:1001900097B944240027112778948895FECFF894C6
:0201A000FFCF8F
:02000004008278
:020000007BF98A
:00000001FF
